:020000020000FC
:100000000DC0189518951895189518951895189568
:10001000B1C01895189518951895D0C000E00EBF7E
:100020000FED0DBF00E808B901E007B907EC06B90C
:1000300002E001B903E00EBD0DEF0DBD0FE80CBDF0
:1000400001E00CB94FEE00EF0ABB0BBB07E007BBAA
:10005000DD27C4E000E3402E502E602E702E7894F1
:10006000EE24FF2420E4339A4FD097FF03C09F77FC
:10007000369AFACF2223C1F73398F694E794F69490
:10008000E794F694E794E0E6F0E0052F000FE00F28
:10009000E192F0825395583008F05527E0E6FF27AB
:1000A000FF24EE2422270191E00E0191F01E2395FA
:1000B0002830C8F3F694E794F694E794F694E7941E
:1000C00004E713E131D026941794079426941794EB
:1000D0000794269417940794F12CE02C32D0A4E0D6
:1000E000BB27022D0F70002319F40FEF0D9301C0F1
:1000F00011D0012D029590640DD09F7B012D0AD067
:10010000002D029507D0ACCF00E205BF88950027EF
:1001100005BF0895E8ECF1E00F70E00FFB1F0491BC
:1001200096FD0F7D0D930895222420E116950795E5
:1001300010F41E0C2F1C2794179407942A95B1F7DE
:10014000089520E1222411240024FF27EE0CFF1C37
:10015000001C111C221C2A9509F40895E3E0029169
:100160000D5F03FD00830081005D07FD0083E0302B
:10017000B1F7ECCF0F930FB70F930DEF0DBD0FE855
:100180000CBD0BB3006F0BBBC298099138E0C0984F
:10019000000F10F4C19A01C0C198C09A3A95B9F7FE
:1001A000C29A0BB3006F04230BBB440F10F04FEE49
:1001B000C4E090680F910FBF0F91189504B1E00E45
:1001C00005B1F01E2A95189530F32AA2E1A424F275
:0201D00020A06D
:00000001FF
